:1000000058C0F2C16FC06EC06DC06CC06BC06AC01A
:1000100069C068C067C066C065C064C063C062C0B4
:1000200061C060C05FC00403090422037700770049
:1000300077002E0072006500630075007200730087
:1000400069006F006E002E006A00700010035500FA
:10005000530042002D003200330032001201100123
:1000600002000008C016E1050001010200010902BA
:100070004300020100803209040000010202010075
:1000800005240010010424020205240600010524B1
:10009000010301070583030800FF09040100020AA8
:1000A00000000007050102080000070581020800A2
:1000B000000011241FBECFEDCDBF10E0A0E6B0E0E0
:1000C000E8EFF7E002C005900D92A236B107D9F72C
:1000D00010E0A2E6B0E001C01D92A23CB107E1F73A
:1000E00003D388C38DCF85B7826085BF8BB780640B
:1000F0008BBF8BE480938C008093B7008AE580935C
:100100008B008093B60008951F93DC01162F809119
:10011000B60084FF07C08091B70098E889278093D4
:10012000B70003C08AE58093B600912FE8EBF0E0BA
:100130008D91819391501916DCF388EB90E0612F3B
:100140004FD11C5F1093B6001F9108951F93DC01DF
:10015000162F80918B0084FF07C080918C0098E857
:10016000892780938C0003C08AE580938B00912FB0
:10017000EDE8F0E08D91819391501916DCF38DE854
:1001800090E0612F2DD11C5F10938B001F9108957B
:100190001F93CF93DF9360919C00635067FDA1C0D4
:1001A00080919900CCE0D0E0C81BD109C056DF4F48
:1001B00080919800803118F4CE0181D28CC08D32AC
:1001C00009F089C0683009F086C083EC80937F0015
:1001D0008AE580936000109262008881807621F029
:1001E000CE0161D2282F65C09A8110928800898142
:1001F000882321F41092890022E054C0853019F43C
:1002000090939D004EC08630B1F58B81813041F4D2
:100210008CE590E090939B0080939A0022E127C0A8
:10022000823021F4CE012AD2282F21C08330F1F46C
:10023000992341F486E290E090939B0080939A008A
:1002400024E015C0913041F48AE290E090939B0045
:1002500080939A0022E20BC0923041F48CE490E04B
:1002600090939B0080939A0020E101C020E080E4FD
:10027000809362001EC0883021F421E08FE990E075
:1002800013C0893019F490939F000BC08A3011F489
:1002900021E008C08B3029F48BE480938C0080939C
:1002A000B70020E088E890E090939B0080939A004C
:1002B00009C02F3F39F4888187FD2E8180E8809323
:1002C000620006C08F81882319F48E81821708F09E
:1002D000822F8093610080919C00181614F4109274
:1002E0009C008091600084FF58C0809161008F3F26
:1002F00009F453C0182F893008F018E0811B80934F
:10030000610080917F0098E8892780937F00112306
:1003100091F18091620087FF08C080E890E0612F32
:100320003FD2182F893098F526C020919A0030913D
:100330009B0086FF0DC0A0E8B0E080E090E0F901EE
:10034000E80FF91FE491ED9301961817C1F708C063
:10035000D901912FE0E8F0E08D9181939150E1F780
:100360001150812F90E01F5F0196820F931F909391
:100370009B0080939A0080E890E0612F31D0612F3C
:100380006C5F6C3041F08FEF8093610004C08FEFA1
:10039000809361006EE16093600094E180B38C70A3
:1003A00031F49150D9F710929D0010929700DF918F
:1003B000CF911F910895A82FB92F80E090E041E0E0
:1003C00050EA60956F5F58F42D9138EF822797952A
:1003D000879510F0842795273F5FC8F3F3CF0895E2
:1003E000EADF8D939D930895CF93CFB7CF93C395B5
:1003F000839BE9F7839B09C0839B07C0839B05C050
:10040000839B03C0839B01C0A6C0DF93C09199006A
:10041000DD27C056DF4F839B02C0DF91EBCF2F93C8
:100420000F931F9300B32FEF03FB20F94F933F93DC
:1004300010B34FEF012703FB21F93BE031C04E7FA2
:10044000012F10B3216028C0102F4D7F22600000C3
:1004500000B329C04B7F2460012F000010B32BC0D4
:1004600010B3477F28602AC04F7E00B320612CC0A4
:100470004F7D10B320622FC04F7B00B3206432C089
:10048000422700B349934FEF0000102713FB20F9D8
:1004900010B31C70C9F1297F91F2012703FB21F9E8
:1004A00000B3237F89F2315058F1102713FB22F952
:1004B00010B3277E79F2012703FB23F92F7C81F209
:1004C00000B3102713FB24F92F7971F200C010B389
:1004D000012703FB25F92F7359F200C000B3102741
:1004E00013FB26F9223040F200C010B3012703FBB2
:1004F00027F9243028F64F77206810B30000F9CF91
:1005000010E41ABF00271CC03B503195C31BD040DC
:1005100010E41ABF0881033C11F10B3401F1209162
:1005200097001981110F1213EDCF4A81441F09362C
:1005300069F10D3211F0013E29F74F7009F0042FD7
:1005400000939E003F914F911F910F912F91DF914A
:10055000CAB7C6FD4CCFCF91CFBFCF911895209190
:100560009E00222379F310919C001123D1F53430A1
:10057000D2F100938A0030939C0020939800109150
:1005800099003BE0311B309399002DC000919C00F5
:1005900001303CF50AE54F7049F43091600034FDBC
:1005A00024C000936000CFE7D0E023C0433049F07F
:1005B00030918B0034FD19C000938B00CCE8D0E063
:1005C00018C03091B60034FD10C00093B600C7EBE0
:1005D000D0E00FC02795A8F45150A9F4220F0000D5
:1005E000F9CF4AE503C042ED01C0432FC4E1D0E09A
:1005F00032E011B31C60939A11BB02B320E41CE0FB
:100600005F93012756E002BB279520F4515021F457
:10061000220FF9CF012756E000003B5A02BBD0F26F
:10062000279528F4515029F4220F0000F9CF012713
:1006300056E0279502BB20F4515021F4220FF9CF48
:10064000012756E02991332302BB21F6037F109145
:100650009D00110FC651D04002BB11F010939700BE
:1006600010E41ABF086011B3137F402F437F5F91DE
:1006700000C000C002BB11BB42BB64CFFC01838140
:10068000813049F48CE590E090939B0080939A0030
:1006900080915C0008958EE690E090939B0080939B
:1006A0009A0083E40895FC0180818076803229F4E9
:1006B0008181813211F48FEF089580E00895DC018B
:1006C000662389F090917D00E92FF0E0E459FF4F17
:1006D0008D9180839F5F9F706150B1F790937D00F3
:1006E0008FEF80939C00089583EF82BB8CE081BBE9
:1006F00090E003C0A8958150E9F7915011F080E097
:10070000FACF11BAF0DC7894A89542DD5D9B10C059
:1007100090917E0080917D00891751F0E92FF0E0E3
:10072000E459FF4F80818CB99F5F9F7090937E004A
:1007300080919C0087FF0DC080917D0090E020910A
:100740007E00821B91098F709070089714F41092AC
:100750009C005F9B0DC090917C00983048F48CB158
:10076000E92FF0E0EC59FF4F80839F5F90937C006E
:1007700080918B0084FFC8CF60917C00662329F4B0
:1007800080916300882309F4BFCF84E690E0DEDC2B
:1007900080917C0088708093630010927C00B4CFBD
:1007A000FC011AB892E09BB982B3806382BB80B32C
:1007B0008073803231F480E789B992B920E699E0FC
:1007C0000DC0803131F486E289B912B820E096E993
:1007D00005C08BE989B912B820E895E288E18AB9A9
:1007E00020839183128213821482158288E086838B
:0807F00087E00895F894FFCFA3
:0207F8005AFFA6
:00000001FF
